:020000040000FA
:0200000079285D
:080008000C2982071E3420348C
:100010001D3420341F3420341F34203420341F3446
:1000200020341F342034820000340134023403347D
:1000300004340534063407340834093410341134D8
:100040001234133414341534163417341834193464
:1000500020342134223423342434253426342734E4
:100060002834293430343134323433343434353470
:1000700036343734383439344034413442344334FC
:100080004434453446344734483449345034513488
:100090005234533454345534563457345834593414
:1000A0006034613462346334643465346634673494
:1000B0006834693470347134723473347434753420
:1000C00076347734783479348034813482348334AC
:1000D0008434853486348734883489349034913438
:1000E00092349334943495349634973498349934C4
:1000F000FF3483018B018A01810191018F018E01FF
:100100008501860187019F019E0183163F3085008E
:100110000030860000308700823081000E309F0062
:100120009E013F309200831281309F000430920084
:100130003C30970040309500203084008001840AD4
:10014000841F9E28051939178519B9173908C03930
:10015000C03C03193A161630E9003B30EA00033080
:10016000E7000130E8000030E1000030E2000C3030
:10017000E3000030E6000130E5000130E400A0308B
:100180008B0083160C108C1083128518D828391A0E
:10019000CB283916CC283912BC14391ED428B916EC
:1001A0008A11BE23BC10F228B9128A117E23BC101A
:1001B000851AF228B91AF22832306102031DE728A5
:1001C000391AF2283916BC148A11BE23BC103730F4
:1001D0006102031DF228391EF2283912BC148A115B
:1001E0007E23BC103C1CFC280A305D020319FA284F
:1001F0008715FC283C10871100305E02031DC528BE
:10020000DF0A00305F02031DC528DF011F151F191B
:1002100007291E089500C528F000030E8301F10090
:100220000A08F2008A01DE0ADB0ADC0ADD0A3A1C4F
:100230001B293A1020293A148A112B218A116C2289
:100240008A11F9228B018B1672088A00710E8300C5
:10025000F00E700E0900B00F39293A303202031D3A
:100260003329BA1EBA15FF30B200BA12BA10BA1347
:1002700008000508F300731A5A29BA1C0800BA10BE
:1002800020303102031C4E2926303102031C522932
:100290003A303102031852293A15562911303102E9
:1002A00003185529BA163A1308003A11B20A8A11EE
:1002B0007B210800BA1C5E29B10A6229BA14BA1758
:1002C000B101B001BA1D0800BA1A7729E0013A1746
:1002D0003A1E70296B29BA11B9148A113622080006
:1002E000BA11B914B91979298A110C2208003A13E4
:1002F0000800B914080014303202031D8E293A1D7B
:10030000092A3B14BB103B11BB113B123B13B30139
:10031000B401B501B601B701B80108003B1CA22920
:100320003A1D95290314B30A96290310B40C1C3006
:100330003202031D0800B30C0318092A3B10BB143A
:10034000B3010800BB1CB7293A1DA9290314B30A3D
:10035000AA290310B50C23303202031D0800B30C88
:100360000318092AB50CBB103B15B30108003B1D4F
:10037000C9293A1DBE290314B30ABF290310B60CBC
:1003800029303202031D0800B60CB60C3B11BB1617
:100390000800BB1ED8293A1DD0290314B30AD1295D
:1003A00003102C303202031D0800BB12BB150800DD
:1003B000BB1DEB293A1DDF290314B30AE029031002
:1003C000B70C31303202031D0800B70CB70CB70C64
:1003D000BB113B1608003B1EFB293A1DF2290314F2
:1003E000B30AF3290310B80C39303202031D080098
:1003F0003B123B1708003B1F08003A1D022A03145A
:10040000B30A032A0310B30C0318092A3B13B301E0
:100410000800BA163A1308003908C039403C0319DD
:10042000172A3908C039803C0319272A362AE101E6
:10043000C001C1010F303505EE000330B50E3505A2
:10044000EF008A110424E3000130E302432AE101B2
:10045000C001C1010F303505EE000330B50E350582
:10046000EF008A110424013EE300432AE101C001A8
:10047000C1010F303505EE000330B50E3505EF0034
:100480008A110424E3000F303405EE000730B40E67
:100490003405EF008A110424E2000F303605EE0027
:1004A0000330B60E3605EF008A110424E4000F3045
:1004B0003705EE000130B70E3705EF008A1104242E
:1004C000E5000F303805EE000F30B80E3805EF00AC
:1004D0008A110424E6000800E00A6008FA3C031DC3
:1004E0000800E0013915E10A61083C3C031D0800E1
:1004F000E1013914E20A62083C3C031D0800E201F4
:10050000E30A3C14DD016308183C031D0800E30105
:10051000660803390319BB17E40A6508023C031D8A
:10052000952ABB1F952A0039962A65088A1105204D
:100530006402031D08000130E400E50A65080D3C73
:10054000031D08000130E500E60ABB136608033905
:100550000319BB1708006108BD008A110E243E086C
:10056000C0003F08C1006208BD008A110E243E0889
:10057000C2003F08C3006308BD008A110E243E0874
:10058000C4003F08C500BC1808004008D00041085E
:10059000D1004208D2004308D3004408D4004508E3
:1005A000D50008006608BD008A110E243E08CA0066
:1005B0003F08CB006508BD008A110E243E08C80024
:1005C0003F08C9006408BD008A110E243E08C60019
:1005D0003F08C700BC1808004A08D0004B08D100EB
:1005E0004808D2004908D3004608D4004708D5007F
:1005F0000800391E002B8A11D2228A110523080017
:100600008A11AB228A11052308000630590203190A
:10061000D90186130608F039F3005908503E8400CA
:10062000000873068600D90A07088F39F300590EAF
:10063000730687008617391E202B061F06172D2BE1
:10064000391D2C2B061F0617DA0A96305A02031D95
:100650002D2B3911061B0613DA01BA1C322B861E0C
:10066000352B372B861A8612372B861E8616391C99
:10067000422B3A1A422B8A115E23B91D422B061EC9
:1006800006164B2BB9194B2BBA1F492B061A06120B
:100690004B2B061E0616BA1E512B071C0714871378
:1006A0000800071807103A1F5B2BBA195B2BB9100B
:1006B000871F87170800871B8713080039106A08EF
:1006C00062026908031C690F63020318692B6B142B
:1006D0006A2B6B10680862026308031C670F6302D1
:1006E0000318732B752B6C14762B6C106C086B0530
:1006F00003197C2BB9110800B91508000F30D00080
:10070000D100D200D300D400D5008A11FE238A1173
:10071000FE234508D0008A11FE234508D100440875
:10072000D0008A11FE234508D2004408D1004308B6
:10073000D0008A11FE234508D3004408D2004308A4
:10074000D1004208D0008A11FE234508D400440895
:10075000D3004308D2004208D1004108D0008A11DA
:10076000FE234508D5004408D4004308D3004208BE
:10077000D2004108D1004008D00008000F30D0005E
:10078000D100D200D300D400D5008A11FE238A11F3
:10079000FE234708D0008A11FE234708D1004608EF
:1007A000D0008A11FE234708D2004608D10049082C
:1007B000D0008A11FE234708D3004608D20049081A
:1007C000D1004808D0008A11FE234708D40046080B
:1007D000D3004908D2004808D1004B08D0008A1144
:1007E000FE234708D5004608D4004908D30048082E
:1007F000D2004B08D1004A08D0000800DB012330AA
:100800005B02031DFF2B08006E086F180A3EEF18ED
:10081000143E6F19283EEF19503E08001330013E78
:100820003D07F40000300318013E8A0074081320CD
:10083000ED006D0E0F39BF006D080F39BE000800C6
:02400E00313F40
:00000001FF
